:04000000B201FE2823
:10000800B216B21EB21232190E28FE39B3003215DA
:100018000310F928321A1628A60032162D200318C4
:100028001B282608342003181B28B21EF92826206E
:100038004B2032113212B21136088400340884176A
:1000480080042C283608840034098005841780052C
:10005800080020204B20262047203308B2190138F9
:10006800A2000830A300A20D03182020031C26209C
:100078004B204720A30B372820204B20360884002C
:1000880034080005FF3E3708840035092928370859
:100098008400350823280408A60036088400803028
:1000A800B3050830A70003100318B30A6920A60C8B
:1000B800A70B58280000AB1A330C6920FC20031446
:1000C80069202F08A3002E08BC288413AB1F7828AA
:1000D800000834042B1F34068000841700083404F9
:1000E800031C34068000832800083404031C3406EB
:1000F8002B1B3406800084173409800583282B08BD
:100108001F39003EA1002A080E3E0318A10A00006C
:10011800C928B31329080319B3170530A8002730D5
:10012800A3001030A3200330A300E830A320A301CC
:100138006430A320A3010A30A3202408AA28A2001F
:100148002508A1002408A000D8202008A000A803A2
:100158000319B31329080319B4282802031808003F
:100168002008031DB313B31B0800303EF428A30175
:10017800A200FF30A207031CA307031CF9280330C1
:10018800A100E630C920BD28A101FC3EA000A109BC
:10019800031CD428FF300000A0070318CF28A007AD
:1001A8006400A10FCE280800A501A4011030A60004
:1001B800210DA40DA50D2208A4022308031C230F5A
:1001C800A5020318EE282208A40723080318230F02
:1001D800A5070310A00DA10DA60BDC282008F928FF
:1001E800840031088A0030088200831303138312C5
:1001F80064000800831607309F0083120730B6009A
:100208004030B4002030AA00AB01AE01AF014C3041
:100218008A0150206F308A01502061308A015020B5
:1002280064308A01502069308A0150206E308A017A
:10023800502067308A01502020308A0150204530F4
:100248008A01502045308A01502050308A015020C0
:1002580052308A0150204F308A0150204D308A0197
:1002680050202C308A01502020308A0150207030D4
:100278008A0150206C308A01502065308A01502054
:1002880061308A01502073308A01502065308A011C
:10029800502020308A01502077308A015020613068
:1002A8008A01502069308A01502074308A01502018
:1002B8002E308A0150202E308A0150202E308A019B
:1002C80050202E308A0150200A308A0150200D30EB
:1002D8008A015020BE01BF01B801B9010730B6003C
:1002E8004030B4002030AA00AB01AE01AF0141306C
:1002F8008A01502064308A01502064308A015020DD
:1003080072308A01502065308A01502073308A018A
:10031800502073308A0150203A308A01502005302D
:10032800A9003808A4003908A5004F30B000B10171
:100338008A018D200A308A0150200D308A01502010
:10034800BE016400F0303E028A110A1203182A2BFB
:100358003E08EF3C8A110A12031CF12A8A110A127C
:10036800B921BF008A110A12F12A02308A003E0818
:02037800002A59
:1004000082070034003400340034003400340034F7
:100410000034003400340034003400341F34FF341E
:10042000B03400340034003400340034003400347C
:10043000003400340034003400340034003400341C
:10044000003400340034003400340034003400340C
:100450000034003400340334F0342F347C3400345E
:1004600000340034003400340034003400340034EC
:1004700000340034003400340034003400340034DC
:1004800000340034003400340034003400340034CC
:1004900000341E341A34003477348034003400348D
:1004A00000340034003400340034003400340034AC
:1004B000003400340034003400340034003400349C
:1004C0000034003400340034003400340034E034AC
:1004D00062340434DF3470340034003400340034C7
:1004E000003400340034003400340034003400346C
:1004F000003400340034003400340034003400345C
:100500000034003400340034033406340034FF3443
:10051000FF348C34003400340034003400340034B0
:10052000003400340034003400340034003400342B
:10053000003400340034003400340034003400341B
:10054000003400340C340E3400343F345F34C33490
:1005500000340034003400340034003400340034FB
:1005600000340034003400340034003400340034EB
:1005700000340034003400340034003400340034DB
:10058000303414340034F034CB34C034C03400344C
:1005900000340034003400340034003400340034BB
:1005A00000340034003400340034003400340034AB
:1005B00000340034003400340034003440343E341D
:1005C0008F3442346F34E03420340034003400344B
:1005D000003400340034003400340034003400347B
:1005E00000340730B6001030B4000730B7000830D0
:1005F000B500A0308A01062039088A010620380893
:100600008A0106203F088A01042005308A01BB20A8
:100610000730B6004030B4002030AA00AB01AE0174
:10062000AF010530A9003808A4003908A5004F30F3
:10063000B000B1018A018D200A308A0150200D30AE
:100640008A015020B80A0319B90ABE0A8A110A128F
:10065000031DA529BE016400F0303E028A110A1272
:1006600003182A2D3E08EF3C8A110A12031CF12CB4
:100670008A110A123F23BF008A110A12F12C04309A
:060680008A003E08002C78
:1008000082070334C034F8347034E734E134F03410
:1008100000340034003401348034BF347F348834F1
:10082000F734E03418340034003400340034003439
:100830000034003400340034003400340034073411
:10084000E134FC347034E734F334F83400340034E9
:10085000003402340034E5343F344734F734F034A4
:1008600004340034003400340034003400340034E4
:10087000003400340034003400340E347334DE3479
:100880007934E73473349834003400340034043459
:1008900001349434B8341C347F34FC3402340034D2
:1008A00000340034003400340034003400340034A8
:1008B0000034003400340E3403348E347934E73499
:1008C000733487341D34F03400340834033408346E
:1008D000023420343E348434013400340034003493
:1008E0000034003400340034003400340034003468
:1008F00000340E3403348E3469346734F134F33405
:100900001B349834003410340134C134E8340134D9
:100910003C343E340034803400340034003400343D
:1009200000340034003400340034003400340E3419
:1009300003348E346F346734E034FB34BB34C0345A
:10094000003420340334903480344E347B34823489
:1009500000344034003400340034003400340034B7
:10096000003400340034003400340E3463348E34E8
:100970006F34673400343B34B934F03400344034DD
:100980000334C834803418347C34DF3400342034E9
:1009900000340034003400340034003400340034B7
:1009A0000034003400340E347334DE34663467347B
:1009B00003343934B0347834003480340334B234FE
:1009C000DF347C347634E3340034103400340034C3
:1009D0000034003400340034003400340034003477
:1009E00000340730B6001030B4000730B7000830CC
:1009F000B500A0308A01062039088A01062038088F
:100A00008A0106203F088A01042005308A01BB20A4
:100A10000730B6004030B4002030AA00AB01AE0170
:100A2000AF010530A9003808A4003908A5004F30EF
:100A3000B000B1018A018D200A308A0150200D30AA
:100A40008A015020B80A0319B90ABE0A8A110A128B
:100A5000031D2B2BBE016400F0303E028A110A12E6
:100A600003182A2F3E08EF3C8A110A12031CF12EAC
:100A70008A110A123F25BF008A110A12F12E063090
:060A80008A003E08002E72
:100C000082070734E134FC34663467340334F93442
:100C1000F3343834003480340334D934FD34F434BC
:100C20007734FF34003410340034003400341C3482
:100C30000334C334F034003400340034003403345B
:100C4000C034F834663467340134F034E134F034BD
:100C5000013400340334FC347F34FB34F134873402
:100C6000003408340034003400341C340734E334D6
:100C7000F8340034003400340034003400340034DC
:100C80000034003400340034E034003401340034E3
:100C90000734FA34F334F4340034FF3400340834C5
:100CA0000034003400341C340E3473349C3400346B
:100CB0000034003400340034003400340034003494
:100CC00000340334E0340034023400340734B934DF
:100CD0004034003400347F34803404340034003431
:100CE00000341C340E3403349C340034003400349B
:100CF0000034003400340034003400340034033451
:100D0000C0340034043400340734F8344034003440
:100D100000341F34003402340034003400341C34F6
:100D20000E3403349C340034003400340034003476
:100D30000034003400340034003400340034003413
:100D4000043400340734B0344034003400343F34C9
:100D5000003402340034003400341C340E340334C4
:100D60009C34003400340034003400340034003447
:100D700000340034003400340034003404340034CF
:100D80000734703400340034003403340034023447
:100D90000034003400341C340E3463349C3400348A
:100DA00000340034003400340034003400340034A3
:100DB0000034003400340034083400340734103474
:100DC0000034003400340B34003401340034003477
:100DD00000341C340E3473349C340034003400343A
:100DE00000340730B6001030B4000730B7000830C8
:100DF000B500A0308A01062039088A01062038088B
:100E00008A0106203F088A01042005308A01BB20A0
:100E10000730B6004030B4002030AA00AB01AE016C
:100E2000AF010530A9003808A4003908A5004F30EB
:100E3000B000B1018A018D200A308A0150200D30A6
:100E40008A015020B80A0319B90ABE0A8A110A1287
:100E5000031D2B2DBE016400F0303E028A150A12DC
:100E600003182A293E08EF3C8A150A12031CF128B0
:100E70008A110A123F27BF008A150A12F12808308A
:060E80008A003E08002874
:1010000082070034003400340034003400340034EB
:1010100000340034083400340E340034003400341A
:1010200000340734003401340034003400341F34F9
:10103000C734E334F834003400340034003400346E
:101040003F3400340034003438341C34003400346D
:10105000083400340E3400340034003400340F34CB
:10106000003401340034003400341F34C334C3343A
:10107000F034003400340034003400347F348034E1
:101080000034003438341C3400340034103400345C
:101090000E3400340034003400340F340034003493
:1010A0008034003400340034003400340034003420
:1010B0000034003400340034F3348034003400341D
:1010C0003834003400340034103400341E3400341A
:1010D0000034003400340D340034003480340034E3
:1010E0000034003400340034003400340034003460
:1010F00000340034E0343B347E3477343B349C3469
:1011000078340034103400341634003400340034A1
:1011100000340334003400348034003400340034AC
:10112000003400340034003400340034003400341F
:10113000E734BE34FF347F34BF34DC34FC34003455
:1011400010340034D6340034003400340034173402
:10115000003400348034003400340034003400346F
:10116000003400340034003400340034E734B83440
:10117000E7347334B934DD34CE3400341034003401
:10118000E63403343834003400341B340034003483
:10119000803400340034003400340034003400342F
:1011A0000034003400340034E334B8341F34733472
:1011B000B934DD34C0340034103401345C340034CC
:1011C0007C34003400340F34003400348034003474
:1011D0000734FE343C343C340F340F340334C03411
:1011E00000340730B6001030B4000730B7000830C4
:1011F000B500A0308A01062039088A010620380887
:101200008A0106203F088A01042005308A01BB209C
:101210000730B6004030B4002030AA00AB01AE0168
:10122000AF010530A9003808A4003908A5004F30E7
:10123000B000B1018A018D200A308A0150200D30A2
:101240008A015020B80A0319B90ABE0A8A110A1283
:10125000031D2B2FBE016400F0303E028A150A12D6
:1012600003182A2B3E08EF3C8A150A12031CF12AA8
:101270008A150A123F21BF008A150A12F12A0A3084
:061280008A003E08002A6E
:1014000082070034F334B834E7347334B934DD344C
:10141000CE3400341034003486340034C034003408
:101420007F34073400340034803400340734FE3411
:101430007E347E341F349F348734E03400340034EB
:101440007F34B834FF347F34B934DC34FC340034B6
:101450001034003496340734FE340034FB340F3437
:10146000003400348034003408347034EE3477347F
:101470003B349D34CE347034003400343E34383440
:10148000773477343934DC34783400341034003431
:1014900046340F34C9340134B0340734A034003436
:1014A00087343934C8347034E03477343834013414
:1014B000CE3400340034003400340034003470344E
:1014C000003400340034003410340034DC3401348F
:1014D000E5340334FE340E340034003483343934BC
:1014E00088347034EC347F343B3403348E3400342D
:1014F00000340034003400340034703400340034DC
:10150000003400341034003416340034DC34043435
:10151000D7340434E03400348334BB349034703432
:10152000FE3437343F3483348E3400340034003496
:10153000003400340034703400340034003400349B
:10154000103400347634023400340534E2340B3481
:10155000003400348334AB3490347034EE340734C8
:101560003B348134CE3460340034003400340034F1
:1015700000340034003400340034003408340034C3
:1015800036340034003408343C340A340034013436
:101590000134EF3410347034EE3477343B349D34FE
:1015A000CE3470340034003400340034003400345D
:1015B000003400340034003408340034263400345D
:1015C0000034083440340F34203401340134C7343B
:1015D000203470347E347E341F349F348734E034BA
:1015E00000340730B6001030B4000730B7000830C0
:1015F000B500A0308A01062039088A010620380883
:101600008A0106203F088A01042005308A01BB2098
:101610000730B6004030B4002030AA00AB01AE0164
:10162000AF010530A9003808A4003908A5004F30E3
:10163000B000B1018A018D200A308A0150200D309E
:101640008A015020B80A0319B90ABE0A8A150A127B
:10165000031D2B29BE016400F0303E028A150A12D8
:1016600003182A2D3E08EF3C8A150A12031CF12CA0
:101670008A150A123F23BF008A150A12F12C0C307A
:061680008A003E08002C68
:10180000820700340334F0340034003400340034F0
:1018100000340034083400340E3400340034003412
:1018200038340C34C03401340134C73420347034BB
:101830003C343C340F340F340334C03400340034AF
:101840000334F834003400340034003400340034FD
:1018500004340034023400340034003400340D34D5
:1018600000340234003400340034003400340034D6
:1018700000340034003400340034003403349C3429
:1018800000340034003400340034003404340034B4
:10189000003400340034003400340734803402341F
:1018A0000034003400340034003400340034003498
:1018B000003400340034003403349C3478347634FB
:1018C000E134E03400340034043400340C340034A7
:1018D0000034003400341D34003402340034003449
:1018E0000034003400340034003400340034003458
:1018F0000034003403349C34FC347F34F334F0344B
:101900000034003402340034003400340034103425
:101910000034113400340434003400340034003412
:101920000034003400340034003400340034003417
:1019300003349D34CE347734773438340034003473
:1019400001340034003400340634143400340234DA
:1019500000340834003400340034003400340034DF
:1019600000340034003400340034003403349D3437
:10197000FE347734773438340034003401340034A2
:10198000023400342134E834003424340034083480
:1019900000340034003400340034003400340034A7
:1019A000003400340034003403349D34C0347734C0
:1019B0007734383400340034003480340034013457
:1019C000C034003400342C3400341034003400347B
:1019D0000034003400340034003400340034003467
:1019E00000340730B6001030B4000730B7000830BC
:1019F000B500A0308A01062039088A01062038087F
:101A00008A0106203F088A01042005308A01BB2094
:101A10000730B6004030B4002030AA00AB01AE0160
:101A2000AF010530A9003808A4003908A5004F30DF
:101A3000B000B1018A018D200A308A0150200D309A
:101A40008A015020B80A0319B90ABE0A8A150A1277
:101A5000031D2B2BBE016400F0303E028A150A12D2
:101A600003182A2F3E08EF3C8A150A12031CF12E98
:101A70008A150A123F25BF008A150A12F12E0E3070
:061A80008A003E08002E62
:101C0000820700340334F834FE3477347334F0340C
:101C100000340034003480340134003400340034A3
:101C20008034203400341034003400340034003464
:101C30000034003400340034003400340034003404
:101C40000334F0347C3477347134E03400340034BD
:101C50000034403401340034E03400344034403443
:101C600000342034003400340034003400340034B4
:101C700000340034003400340034003400340034C4
:101C80000034003400340034003400340034203494
:101C9000003400343F34093440344034003440349C
:101CA0000034003400340034003400340034003494
:101CB0000034003400340034003400340034003484
:101CC00000340034003400340034103400348034E4
:101CD0001C342F3400348034003480340034003419
:101CE0000034003400340034003400340034003454
:101CF0000034003400340034003400340034003444
:101D000000340034003408340034403420341834B3
:101D100000348034013400340034003400340034A2
:101D20000034003400340034003400340034003413
:101D30000034003400340034003400340034003403
:101D400000340434003460341734F0340134003487
:101D500002340034003400340034003400340034E1
:101D600000340034003400340034003400340034D3
:101D700000340034003400340034003400340234C1
:101D8000003430340834083402340034043400346D
:101D900000340034003400340034003400340034A3
:101DA0000034003400340034003400340034003493
:101DB00000340034003400340034013480340834FA
:101DC0000434103404340034183400340034003443
:101DD0000034003400340034003400340034003463
:101DE00000340730B6001030B4000730B7000830B8
:101DF000B500A0308A01062039088A01062038087B
:101E00008A0106203F088A01042005308A01BB2090
:101E10000730B6004030B4002030AA00AB01AE015C
:101E2000AF010530A9003808A4003908A5004F30DB
:101E3000B000B1018A018D200A308A0150200D3096
:101E40008A015020B80A0319B90ABE0A8A150A1273
:101E5000031D2B2DBE016400F0303E028A110A16CC
:101E600003182A293E08EF3C8A110A16031CF128A0
:101E70008A150A123F27BF008A110A16F12810306E
:061E80008A003E08002864
:1020000082070034003400340034003400340034DB
:102010000034003400340034403404340334E034F9
:1020200008340034203400340034003400340034E8
:102030000034003400340034003400340034003400
:1020400000340034003400340034003400340034F0
:10205000003400343034023400340034203400348E
:10206000C034003400340034003400340034003410
:1020700000340034003400340034003400340034C0
:1020800000340034003400340034003400340034B0
:102090000C34013400340034803403340034003410
:1020A0000034003400340034003400340034003490
:1020B0000034003400340034003400340034003480
:1020C000003400340034003400340034033400346D
:1020D0004034033400340C34003400340034003411
:1020E0000034003400340034003400340034003450
:1020F0000034003400340034003400340034003440
:1021000000340034003400340034E034203404342B
:1021100000347034003400340034003400340034AF
:10212000003400340034003400340034003400340F
:1021300000340034003400340034003400340034FF
:102140000034003400341C34183418340334803420
:1021500000340034003400340034003400340034DF
:1021600000340034003400340034003400340034CF
:1021700000340034003400340034003400340034BF
:1021800000340334E134C0347C340034003400348F
:10219000003400340034003400340034003400349F
:1021A000003400340034003400340034003400348F
:1021B000003400340034003400340034003400347F
:1021C0001F34FF34803400340034003400340034D1
:1021D000003400340034003400340034003400345F
:1021E00000340730B6001030B4000730B7000830B4
:1021F000B500A0308A01062039088A010620380877
:102200008A0106203F088A01042005308A01BB208C
:102210000730B6004030B4002030AA00AB01AE0158
:10222000AF010530A9003808A4003908A5004F30D7
:10223000B000B1018A018D200A308A0150200D3092
:102240008A015020B80A0319B90ABE0A8A150A126F
:10225000031D2B2F0730B6004030B4002030AA00F9
:10226000AB01AE01AF010530A9003808A400390860
:10227000A5004F30B000B1018A018D200A308A01DB
:1022800050200D308A01502041308A0150206C309E
:102290008A0150206C308A01502020308A01502061
:1022A00064308A0150206F308A0150206E308A01DC
:1022B000502065308A01502021308A0150200A3098
:1022C0008A0150200D308A01502063008A110A16BD
:0222D00065297E
:02400E00753FFC
:00000001FF
